:02000000E12BF2
:10000800FF00030E8301E4000A08E3008A017B086D
:10001800A2007C08A1007D08A0008B1C22280230C9
:1000280085060230FB008630FC009930FD00FD0B90
:100038001B28FC0B1B28FB0B1B288B102208FB0022
:100048002108FC002008FD0063088A00640E830074
:06005800FF0E7F0E0900FF
:04005E000000080096
:0C0062001030FD00FD0B332800000800EA
:10006E000830FC002330FD00FD0B3B28FC0B3B2829
:02007E00080078
:1000800083160313A01B4728831287114928831264
:1000900087158316201B4F288312071151288312BE
:1000A00007158316A01A5728831287105928831220
:1000B00087148316201A5F28831207106128831281
:1000C00007145E18652807166628071287162F2062
:1000D00087128316A0196F28831287117128831243
:1000E0008715831620197728831207117928831220
:1000F00007158316A0187F28831287108128831282
:1001000087148316201887288312071089288312E2
:1001100007145E188D2807168E28071287162F20C1
:0E01200087125E1C9528372096283120080093
:10012E00710DF80DF90D7408F8027508031C750FA2
:10013E00F902F00DF10D0F30FC00710DF80DF90DF7
:10014E007408701CB028F8027508031C750FF902AC
:10015E00B528F80775080318750FF907F00DF10D9E
:10016E00FC0BA4287018C1287408F807750803182A
:08017E00750FF90700000800ED
:10018600831203135E106F088316A00040205E14CE
:0201960008005F
:1001980083120313FD01F901F801710870040319B2
:1001A800003471087506FA00FA1BFD09FB01F51FFA
:1001B800E228F409F509F40A0319F50AF11FE928F8
:1001C800F009F109F00A0319F10A71087504FA0037
:1001D800FA1BFE2897207B181129FD1F0034F0090F
:1001E800F109F00A0319F10AF809F909F80A0319DB
:1001F800F90A0034F51F0D29F11B09297108F900C6
:100208007008F800F101F001F128F101F001F00A9D
:100218000034F109F009FB0AEE28F80A0319F90A73
:1002280074087802031DF12875087902031DF12866
:10023800F901F801F00A0319F10AF11FF128000089
:04024800FF34080077
:0E024C001930FD00FD0B2829000000000800FD
:0E025A008312031357088A005608820008001A
:100268004629803083120313EB005929C030EB0074
:1002780059299430EB005929D430EB0059298030A2
:10028800EB005929831203136B08013A0319352926
:100298006B08023A03193A296B08033A03193D29F6
:1002A8006B08043A0319402943296C03F0006B08D2
:1002B800F0077008EB0070088316A00040205E105D
:1002C800EE016E086D0784000008031973296E0893
:1002D8006D0784000008EF00C320EE0A65295E144C
:0202E80008000C
:0E02EA00A530FD00FD0B772900000000080084
:1002F800831203132308031DA429E830F4000330F4
:10030800F5005408F0005508F100CC20700871047D
:100318000319A0292508E500E830F4000330F500AA
:100328005408F0005508F100CC203030F00765087B
:10033800840070088000A4292508840020308000EB
:10034800250AE5006430F4000030F5005408F00098
:100358005508F100CC200A30F4000030F500CC201C
:100368007808F0007908F1003030F007650884005B
:100378007008800002302507E5000A30F4000030DC
:10038800F5005408F0005508F100CC200A30F400BC
:100398000030F500CC207808F0007908F100303002
:1003A800F007650884007008800004302507E50020
:1003B8000A30F4000030F5005408F0005508F10048
:1003C800CC207808F0007908F1003030F007650893
:1003D8008400700880000230EB000130EC00250832
:1003E800ED0034212408031D1C2AE830F4000330F2
:1003F800F5005808F0005908F100CC207008710485
:100408000319182A2608E500E830F4000330F5003F
:100418005808F0005908F100CC203030F007650882
:100428008400700880001C2A260884002030800080
:10043800260AE5006430F4000030F5005808F000A2
:100448005908F100CC200A30F4000030F500CC2027
:100458007808F0007908F1003030F007650884006A
:100468007008800002302607E5000A30F4000030EA
:10047800F5005808F0005908F100CC200A30F400C3
:100488000030F500CC207808F0007908F100303011
:10049800F007650884007008800004302607E5002E
:1004A8000A30F4000030F5005808F0005908F1004F
:1004B800CC207808F0007908F1003030F0076508A2
:1004C8008400700880000230EB000A30EC00260837
:0604D800ED0034210800D4
:1004DE008030831203136606F00080307002031D15
:1004EE007A2A003065020318852A6508003CF00060
:1004FE006608031C013EF101F10208006508F000D8
:06050E006608F100080080
:10051400831203136608F1000130F0007108031917
:10052400972AF00D7010FF3E912A7008EA007009B6
:10053400E90065088400E801E7016708073C031C3B
:10054400C32A690880058417690880052F206A0872
:1005540080042F2084136A080005F0000319BF2AC1
:100564006708F1000130F00071080319BD2AF00D8D
:100574007010FF3EB72A7008E80431203120E70AE2
:080584009F2A6808F00008003E
:10058C00831203136608F1000130F000710803199F
:10059C00D32AF00D7010FF3ECD2A7008EA00F00946
:1005AC007008E90065088400700880058417E8016C
:1005BC006808073C031CF82A6808F0006708F1007B
:1005CC0070080319ED2AF10CF113FF3EE72A6908B4
:1005DC008005711CF32A6A08800426216A088004AD
:0C05EC00E80ADE2A8413312031200800C8
:1005F8002D218A110A128000840AD60A0319D70A03
:08060800F003031DFC2A0800A9
:1006100083120313FB01FA01F9018030F800F10C99
:10062000F00C031C1C2B7408F90775080318750FD0
:10063000FA070318FB0A0310F01F242B7408FA07AB
:1006400075080318750FFB07FB0CFA0CF90CF80C76
:10065000031C0F2B7B08F3007A08F2007908F100E5
:060660007808F00008001C
:10066600831203136608F1000130F00071080319C4
:10067600402BF00D7010FF3E3A2B7008E800F00991
:100686006508840070088005841770088005752148
:10069600680880048413262168080005E7006708B7
:1006A600003A013003190030E70075216708F000B1
:0206B60008003A
:1006B8006E2B803083120313E500812BC030E500D8
:1006C800812B9430E500812BD430E500812B8030DC
:1006D800E500812B831203136508013A03195D2B8A
:1006E8006508023A0319622B6508033A0319652B5A
:1006F8006508043A0319682B6B2B6603F00065083C
:10070800F0077008E5005E1470088316A00040200A
:0E0718005E1067088316A00040205E140800E3
:100726008316031387120712071087100711871104
:1007360083128712071287110711871007103720B7
:10074600372037208714071487162F208712372063
:1007560087162F208712372087162F2087123720DB
:10076600071087162F208712372087162F2087120B
:100776008710871587162F208712372087110714B1
:1007860087162F208712071087162F2087123720EB
:1007960087162F208712071487162F2087123720D7
:1007A600071087162F208712871507158714071439
:0C07B60087162F20871237205E140800E1
:1007C20040258316031387010C30850091018312A3
:1007D2008501870107309900932301308316A00019
:1007E20040200C308316A000402085140130EB001D
:1007F2000130EC002730ED0034210630FB001330CD
:10080200FC00AD30FD00FD0B042CFC0B042CFB0B9B
:10081200042C000000000130EB000130EC00373006
:10082200ED0034210230E5000630E600DF30E7005B
:100832005C230230E5000F30E600DF30E7005C2386
:100842000230E5000730E6004330E7005C23023067
:10085200E5001030E6004630E7005C238316810194
:100862008B100B168B1705308312E5000530E6005E
:1008720033230530E5000530E600CC30E700C62220
:100882000530E5000530E6004430E700C6228B174C
:100892000430FB000C30FC003330FD00FD0B4F2C0C
:1008A200FC0B4F2CFB0B4F2C000000000530E50029
:1008B2000530E60033230530E5000530E600CC3094
:1008C200E700C6220530E5000530E600BE30E7004D
:1008D200C6220530E5000530E6008A227008DD00F8
:1008E2000530E5000530E6008A227008DC00700859
:1008F200F500F4015D087407F20075080318013E63
:10090200F3007208DA007308DB00F31F942C013045
:10091200A300250884002D308000DA09DB09DA0AF9
:100922000319DB0A952CA3015A08E1005B08E200D7
:10093200E20CE10CE2135A1CA32C0530DF0000305C
:10094200E000A52CDF01E0016108F0006208F1007F
:100952000A30F4000030F50008235F087007D40065
:1009620071080318013E6007D50023080319F02C13
:100972005408F0005508F1000930F4000030F50089
:1009820008230530F4000030F500CC207008403C0C
:10099200F2007108031C013E013CF3007208D8000A
:1009A2007308D90080307306F00080307002031D96
:1009B200DC2C003072020318EE2C0130A400260851
:1009C20084002D3080005808E5005908E6006F22A7
:1009D2007008D8007108D900EF2CA401062D540824
:1009E200F0005508F1000930F4000030F50008234A
:1009F2000530F4000030F500CC2040307007D800FC
:100A020071080318013E013ED9007C21342C082DC7
:100A800023308400313083120313F0000E30D6007F
:080A90000530D700FC2208002C
:020A1C000034A4
:020A1E000034A2
:020A2000483458
:020A22004E3450
:100A24004C3443344434203449346E34693474349B
:100A3400693461346C3469347A3465346434003430
:100A440052346F346F346D342034543465346D341F
:100A5400703465347234613474347534723465348A
:020A640000345C
:0C0A66003034303430342E34303400345E
:0C0A72003034303430342E343034003452
:02400E00F40FAD
:00000001FF
